:100000000C9437060C9454060C9454060C94540625
:100010000C9454060C9454060C9454060C945406F8
:100020000C9454060C9454060C94462B0C941A2CE5
:100030000C9491250C9454060C9454060C9454067C
:100040000C9454060C9454060C9454060C945406C8
:100050000C9454060C9418260C9454060C945406D4
:100060000C9454060C9454060C9454060C945406A8
:100070000C9454060C9454060C9454060C94540698
:100080000C9454060C9454060C9454060C94540688
:100090000C9454060C9454060C9454060C94540678
:1000A0000C9454060C9454060C94540614001A0034
:1000B00008001500170000001C0018000C001200BA
:1000C000130004001600070009000A0000000B00DE
:1000D0000D000E000F0033001D001B00060019006C
:1000E0000500E0001100100036003700380029003C
:1000F0002B00E300E1002A00E2002C0021522D0039
:10010000340028001E021F0252002F02300200009D
:100110004B0024002500260025022002500051003B
:100120004F00210200004E002100220023002E0279
:100130002F003000260227022402E00035001E00B6
:100140001F002000310002524900E300E1002A00B4
:10015000E2002C000100370027002E0049004A0071
:1001600052004D004B000000520040004100420090
:1001700043004C00500051004F004E000000510061
:100180003D003E003F0044000000A90000000000C8
:10019000007CE00000003A003B003C0045000352B8
:1001A000AA00E300E1002A00E2002C000052460011
:1001B0004700480029001E001F0020002100000009
:1001C0003A003B003C001C00490014001A000800E3
:1001D0001500170000000C00120013004A004B002D
:1001E00004001600070009000A00E100E2004C00CC
:1001F00052004D004E001D001B00060019002C008F
:100200002452E400500051004F0005002300240058
:10021000250026002700000031003E003F0040007E
:1002200041001C0018000C0012002F0000003500D7
:1002300042004300440045000B000D000E000F007B
:1002400033004700000000000000000000000052E2
:100250001100100036000000010000000000000046
:100260000000000044454255473A206469736162CA
:100270006C65642E0A0044454255473A20656E611C
:10028000626C65642E0A006C65645F7461736B3A1E
:1002900020253032580A004F6E6573686F743A201B
:1002A0006163746976653A2025640A000A00253086
:1002B000313662003A200025303258000A722F632E
:1002C00020303132333435363738394142434445B2
:1002D000460A00556E69636F646520696E707574B7
:1002E000206D6F64652073657420746F3A202575E6
:1002F0000A00556E69636F646520696E70757420BD
:100300006D6F646520696E697420746F3A2025757D
:100310000A00313A0964656C6179282A31306D73BD
:10032000293A2025750A323A09696E746572766138
:100330006C286D73293A2025750A333A096D617866
:100340005F73706565643A2025750A343A097469EB
:100350006D655F746F5F6D61783A2025750A353A77
:1003600009776865656C5F6D61785F73706565645A
:100370003A2025750A363A09776865656C5F7469B5
:100380006D655F746F5F6D61783A2025750A007046
:100390003A097072696E742076616C7565730A64CF
:1003A0003A097365742064656661756C74730A75C7
:1003B000703A092B310A646E3A092D310A6C743A8D
:1003C000092B31300A72743A092D31300A455343F2
:1003D0002F713A09717569740A0A73706565642032
:1003E0003D2064656C7461202A206D61785F7370B4
:1003F000656564202A2028726570656174202F204D
:1004000074696D655F746F5F6D6178290A776865DF
:1004100072652064656C74613A20637572736F72E3
:100420003D25642C20776865656C3D25640A53651D
:100430006520687474703A2F2F656E2E77696B692A
:1004400070656469612E6F72672F77696B692F4DD4
:100450006F7573655F6B6579730A004D3E20004DC3
:1004600025753A25733E20003F0A003D2025750A78
:10047000003F0A0064656661756C74730A00257537
:100480000A003F0A000A092D2056616C7565732029
:100490002D0A00710A000A092D204D6F7573656BD6
:1004A0006579202D0A003F00433E20004C25640A58
:1004B000000A092D20537461747573202D0A686F2A
:1004C00073745F6B6579626F6172645F6C6564738E
:1004D00028293A20253032580A6B6579626F61729B
:1004E000645F70726F746F636F6C3A20253032589E
:1004F0000A6B6579626F6172645F69646C653A204A
:10050000253032580A6B65796D61705F636F6E6676
:1005100069672E6E6B726F3A20253032580A746903
:100520006D65725F72656164333228293A20253027
:10053000386C580A002573000A092D20436F6E732A
:100540006F6C65202D0A4553432F713A0971756907
:10055000740A6D3A096D6F7573656B65790A000AE7
:10056000092D204D61676963202D0A443A094465CD
:10057000627567204D65737361676520546F6767A7
:100580006C650A583A094D61747269782044656255
:100590007567204D6F646520546F67676C65202D0B
:1005A0002053686F77206B6579707265737365731C
:1005B00020696E206D617472697820677269640ABF
:1005C0004B3A094B6579626F6172642044656275CC
:1005D0006720546F67676C65202D2053686F772004
:1005E0006B65797072657373207265706F72740ACF
:1005F0004D3A094465627567204D6F7573652054E7
:100600006F67676C650A563A0956657273696F6E53
:100610000A533A095374617475730A433A09416382
:1006200074697661746520436F6E736F6C65204DDD
:100630006F64650A46312D4631303A095377697443
:10064000636820746F204C6179657220302D3920E9
:1006500028463130203D204C30290A302D393A09C6
:1006600053776974636820746F204C6179657220D8
:10067000302D390A47524156453A09537769746318
:100680006820746F204C6179657220302028616C7D
:100690007465726E617465290A423A094A756D7013
:1006A00020746F20426F6F746C6F616465720A45CD
:1006B00053433A094A756D7020746F20426F6F740E
:1006C0006C6F616465722028616C7465726E617410
:1006D00065290A453A095072696E742045455052A1
:1006E0004F4D2053657474696E67730A4241434BE2
:1006F00053504143453A09436C656172204545506A
:10070000524F4D0A4E3A094E4B524F20546F676775
:100710006C650A006B65796D61705F636F6E666909
:10072000672E7261773A20253032580A2E7377612E
:10073000705F636F6E74726F6C5F636170736C6F08
:10074000636B3A2025750A2E636170736C6F636B5F
:100750005F746F5F636F6E74726F6C3A2025750AF9
:100760002E737761705F6C63746C5F6C6775693A48
:100770002025750A2E737761705F7263746C5F72E7
:100780006775693A2025750A2E737761705F6C6111
:100790006C745F6C6775693A2025750A2E737761F2
:1007A000705F72616C745F726775693A2025750AB3
:1007B0002E6E6F5F6775693A2025750A2E73776113
:1007C000705F67726176655F6573633A2025750AAD
:1007D0002E737761705F6261636B736C6173685FC6
:1007E0006261636B73706163653A2025750A2E6ED2
:1007F0006B726F3A2025750A2E737761705F65738F
:10080000636170655F636170736C6F636B3A202521
:10081000750A0064656275675F636F6E6669672E4F
:100820007261773A20253032580A2E656E61626C0B
:10083000653A2025750A2E6D61747269783A202513
:10084000750A2E6B6579626F6172643A2025750AAC
:100850002E6D6F7573653A2025750A006565636FA7
:100860006E6669673A0A64656661756C745F6C618F
:100870007965723A2025750A003F004E4B524F3A77
:10088000206F66660A004E4B524F3A206F6E0A0088
:100890000A6D6F7573653A206F66660A000A6D6FA0
:1008A0007573653A206F6E0A000A6B6579626F6135
:1008B00072643A206F66660A000A6B6579626F613E
:1008C00072643A206F6E0A000A6D61747269783A38
:1008D000206F66660A000A6D61747269783A206F4B
:1008E0006E0A000A64656275673A206F66660A00E0
:1008F0000A64656275673A206F6E0A000A0A4A75D3
:100900006D70696E6720746F20626F6F746C6F61B9
:100910006465722E2E2E2000433E2000436C6561DC
:1009200072696E6720454550524F4D0A00290A00F2
:100930002575002F002575005D2800256400200026
:10094000256400200025640020002564007C00252B
:10095000303258006D6F7573656B6579205B62741A
:100960006E7C782079207620685D287265702F6112
:10097000636C293A205B0000000000000000002AA0
:100980002B28000000000000000000000000000014
:10099000000029000000002C1E34202122243426CF
:1009A00027252E362D3738271E1F202122232425C8
:1009B000263333362E37381F0405060708090A0B7D
:1009C0000C0D0E0F101112131415161718191A1BEF
:1009D0001C1D2F3130232D350405060708090A0B8D
:1009E0000C0D0E0F101112131415161718191A1BCF
:1009F0001C1D2F3130354C000000000000000000AD
:100A000000000000000000000000000000000000E6
:100A100000000000000000000000007E0F00D4FF76
:100A2000FFFFC7000000780A002530325820006E12
:100A30006B726F5F7265706F72743A202530325836
:100A4000207C20000A002530325820006B65796236
:100A50006F6172645F7265706F72743A2025303214
:100A600058207C200064656C5F6B65795F626974F7
:100A70003A2063616E27742064656C3A2025303219
:100A8000580A006164645F6B65795F6269743A203B
:100A900063616E2774206164643A20253032580AFD
:100AA0000073757370656E64696E67206B6579623B
:100AB0006F6172640D0A005B575D005B535D005B04
:100AC000525D005B445D005B435D000E03410074BA
:100AD0000072006500750073000000180354006583
:100AE00000630068006E006F006D0061006E0063BF
:100AF0000079000000040309040902540003010006
:100B0000A0FA0904000001030101000921110100FC
:100B100001224400070581030800010904010001C6
:100B20000300000009211101000122B6000705821F
:100B30000320000109040200010300000009211143
:100B400001000122150007058303200001120100A6
:100B500002000000080912E5A108000102000106D8
:100B600031FF0974A1010975150026FF0095207554
:100B7000088102C005010902A10185020901A10045
:100B8000050919012908150025019508750181023B
:100B90000501093009311581257F95027508810607
:100BA00009381581257F950175088106050C0A38DD
:100BB000021581257F950175088106C0C0050109D0
:100BC00080A101850319012AB700150126B70095F8
:100BD0000175108100C0050C0901A10185041901EE
:100BE0002AA002150126A002950175108100C005FA
:100BF000010906A1018506050719E029E715002569
:100C0000019508750181020507190029EF150025D6
:100C10000195F075018102050819012905950575F1
:100C2000019102950175039101C005010906A10119
:100C3000050719E029E715002501950875018102CE
:100C40009501750881010507190029FF150026FF88
:100C5000009506750881000508190129051500256C
:100C600001950575019102950175039101C011244B
:100C70001FBECFEFDAE0DEBFCDBF12E0A0E0B1E0F3
:100C8000E2E4FEE502C005900D92AE3CB107D9F753
:100C900023E0AEECB2E001C01D92AD3EB207E1F739
:100CA0000E9419180C94992E0C940000FF93EF9356
:100CB000E091CE02F091CF02309709F00995EF91C3
:100CC000FF910895FC018591803011F0EFDFFBCF9B
:100CD0000895FF27E0E230E247FF0CC0419597FFFF
:100CE00009C0EDE26095709580959095611D711D2C
:100CF000811D911D27FF02C0219530E350E2AA27F4
:100D0000660F771F881F991FAA1FA41710F0A41B36
:100D100063955A95A9F7AA3008F0A95FA05DAF9333
:100D2000F395611571058105910541F7ED3211F4D7
:100D3000EF93F395F21718F43F93F395FBCF8F9150
:100D4000B5DFFA95E1F70895E991F9918591803041
:100D500021F0853219F0AADFF9CF089520E0E89458
:100D600055915532C1F3503311F4689455915A336B
:100D700048F4505390F3220F022E220F220F200D21
:100D8000250FF4CF0EF4219589919991533619F3DB
:100D9000533729F1533559F1BC0188279927E89435
:100DA0005C3621F48991999168945591543639F4BF
:100DB00046EF7EF077FF0DC08FEF9FEF0AC05537EB
:100DC0004AE039F0583540E121F0523642E009F06E
:100DD0000895FF93EF937DDFEF91FF91B7CFFF93DE
:100DE000EF93FC0181918030B9F360DFFBCFFF937B
:100DF000EF9368DFF1CFDF93CF93CDB7DEB72596C2
:100E0000A3DFCF91DF9108958530B8F46430A8F462
:100E10004B3098F450E09BE0699F400D511D112428
:100E2000FA019CE2899FE00DF11D1124EE0FFF1FD6
:100E3000E455FF4F85919491089581E090E00895E5
:100E40000E94040708959C013A9521153F4150F5F1
:100E5000FC01EE27F170BC0166277270AC014427DB
:100E600054709C012227387094FF0EC080E1EF2B54
:100E700009F480E0672B09F08062452B09F080645B
:100E8000232B89F08068089581E0EF2B09F480E03E
:100E9000672B09F08260452B09F08460232B19F041
:100EA0008860089580E00895CF93DF93EB010E945E
:100EB0002307FE010995DF91CF910895CF93DF932A
:100EC000EC01805E9109089720F06FEC7CE02097A0
:100ED00011F462E97AE0CE010E9454078C2F0E943F
:100EE0008409DF91CF910895CF93DF93EC010E94A5
:100EF000170ACE01805E9109089720F066ED7CE02C
:100F0000209711F469E97AE0CE010E945407DF913D
:100F1000CF9108950F931F93CF93DF938C01EB0133
:100F20000E945E07209741F4C8010E947407DF9178
:100F3000CF911F910F9108958FE99FE00197F1F7ED
:100F400000C000002197EECF70E060E0893391058A
:100F500011F460E570E00E948A07089581E0089529
:100F60000E94AE07089581E008950E94AE0708959B
:100F70000E94B507089508950E94BB070895A6E052
:100F8000B0E0E5ECF7E00C94F52D49835A839E839D
:100F90003091D50289819A8131111AC03E81332363
:100FA00099F0222389F00E94420E182F682F898120
:100FB0009A810E941E0E69817A81812F0E946B1591
:100FC0002696E3E00C94112E0E94300E182FF3CFDA
:100FD0000E94420E69817A81F1CFFC01262F408167
:100FE000518162817381848195810E94BF07089538
:100FF000CF93DF93EC0161E00E94ED07BE010E94F8
:10100000B007DF91CF910895CF93DF93EC0160E0BB
:101010000E94ED07BE010E94BC07DF91CF910895A9
:1010200021E030E0A90102C0440F551F8A95E2F784
:10103000CA010E94400D0895CF93C82F81E090E02F
:101040000C2E02C0880F991F0A94E2F70E94C41266
:101050008C2F0E941008CF91089581E008950E947E
:101060002D080895CF93C82F0E94F30C8C2F0E9457
:101070002F082FEF84E39CE0215080409040E1F75F
:1010800000C00000CF91089581E00E9432080E94C4
:101090003C26089580E00E9432080E944D26089563
:1010A0000F931F93CF93DF938C0161E00E94ED07B4
:1010B000EC01B8010E94B807811106C080E0DF9101
:1010C000CF911F910F910895B801CE010E9443184E
:1010D0008823A1F3B801CE010E946322882371F313
:1010E000B801CE010E94521D882341F3B801CE0100
:1010F0000E94281D882311F3B801CE010E946D16AD
:101100008823E1F2F8018581882369F0C330FCE788
:10111000DF07A1F160F4C130ECE7DE0789F1C0F42C
:10112000C115DC4791F0C8010E94B307C8CFCB3589
:10113000ECE7DE0759F1CC35FCE7DF0721F1CA35D2
:10114000DC4789F70E949F12EECF0E944408B6CF79
:1011500090919A03892F8E7F90FF816080939A03EC
:1011600080FF09C086E792E09F938F930E94FB0661
:101170000F900F90A3CF84E692E0F6CF0E94A712C3
:101180000E944A089BCF0E949512CDCF0E94A312C5
:10119000CACF0E946D250E940E0908950E9412096F
:1011A0000E9472250895829590E09C01220F331FC2
:1011B000220F331F2C7C9595879595958795837382
:1011C000282B30E0C901880F991F8A7A3595279519
:1011D0002575822B0895CF93DF93D92F0E94D308D2
:1011E000C82F8D2F0E94D3089C2FDF91CF91089597
:1011F00081E008950895CF93DF93D82F0E94F808D7
:10120000C82F882319F08D2F0E94FA088C2FDF91A8
:10121000CF91089508950E94FB08089580E00E94F0
:101220000B0908950E94AC220E940B090895CF93E8
:101230000E94AC22C82F8091D0028C1701F1C0937C
:10124000D0020E94FD256093D1027093D202809358
:10125000D3029093D40280919A038570853061F413
:101260001F92CF9387E892E09F938F930E94FB0693
:101270000F900F900F900F908C2F0E940B09CF9121
:101280000895ADE0B0E0E7E4F9E00C94F62D48876E
:1012900059876A877B878C879D8791110E9492115D
:1012A0001F8286E0FE013896DE01119601900D92B4
:1012B0008A95E1F78D8181110DC029813A814B8199
:1012C0005C816D817E818F810E94D9102D96E2E034
:1012D0000C94122ECE0101960E94F8078111EDCFD9
:1012E000F5CFFC012481213021F4808191810E947D
:1012F000740E0895662329F00E94B31E0E94861F73
:1013000008950E940D1FFACFCF93C82F8823C9F0EC
:101310008238C9F40E94B92281FD13C089E30E947A
:1013200084240E9426122FEF87EE93E02150804004
:101330009040E1F700C0000089E30E949E240E94D3
:101340002612CF9108958338A1F40E94B92280FD1E
:10135000F8CF83E50E9484240E9426122FEF81EEAD
:1013600094E0215080409040E1F700C0000083E508
:10137000E4CF8438A1F40E94B92282FDE2CF87E451
:101380000E9484240E9426122FEF81EE94E02150C7
:1013900080409040E1F700C0000087E4CECF8CEFA2
:1013A0008C0F813A98F48C2F0E94C81C8111C9CFF0
:1013B0008C2F0E94D623882329F08C2F0E949E24F4
:1013C0000E9426128C2F0E948424B9CF80E28C0FB9
:1013D000883048F4C77081E001C0880FCA95EAF7E9
:1013E0000E947211ACCFEBE5EC0FE33040F4F0E07B
:1013F000E05BFE4F808190E00E946A23A2CFE8E587
:10140000EC0FEB3150F4F0E0EE0FFF1FE65EFE4F05
:10141000808191810E948F2394CF83E38C0F83314D
:1014200008F08FCF61E08C2F0E947A098ACF882341
:1014300009F456C0823879F40E94B92281FF50C065
:1014400089E30E9484240E94261289E30E949E243C
:101450000E9426120895833859F40E94B92280FF11
:101460003FC083E50E9484240E94261283E5EECFCC
:10147000843859F40E94B92282FF32C087E40E9466
:1014800084240E94261287E4E1CF9CEF980F913AC2
:10149000E8F290E2980F983050F4877091E001C024
:1014A000990F8A95EAF7892F0E947811D1CF9BE591
:1014B000980F933028F490E080E00E946A2308950A
:1014C00098E5980F9B3128F490E080E00E948F23EC
:1014D000089593E3980F933118F460E00E947A091D
:1014E00008951F93CF93DF93182FEB010E94840977
:1014F000209739F4812F0E94170ADF91CF911F9115
:1015000008958FE99FE00197F1F700C0000021974F
:10151000EFCF70E060E0893311F460E570E00E9485
:10152000710A0895882321F00E9472110E942612E8
:101530000895882321F00E9478110E9426120895B0
:10154000B0E0A0E0E6EAFAE00C94EF2D6C01D62FB3
:10155000C72FFC011581068102950F700E9468114A
:10156000E82E8823F9F0E12E1123E1F08C2F807F03
:10157000803461F080E28D0F883008F18C2F807EFE
:10158000803221F4D230D8F00023C9F08091C80312
:1015900082FF15C082E00E9456120E94681191E0FD
:1015A000E82EE926BC2EB2949FE0B922FBE0FB15A1
:1015B000B8F1EB2DF0E0E556F14D0C94E02DE12C67
:1015C000F1CF0C2F0F70C07F11F00295007F112317
:1015D00099F0002359F080E28D0F883010F0D1117E
:1015E00007C0802F0E9472110E9426128D2F5AC0B0
:1015F000802F0E948511F8CF8D2F0E94170A00239B
:1016000079F080E28D0F883010F0D11104C0802F66
:101610000E94781103C0802F0E948B110E94261215
:10162000EB2DE850FF0B349720F40E94AC220E946F
:101630000B09EE2089F00E94641180FD0DC0F601B7
:1016400015820E945E110E947C0DC6010E94AC0CA6
:101650000E945E110E948C0DCDB7DEB7E9E00C94BC
:101660000B2E2C2F2F70F22EC07FC03219F0F29467
:1016700080EFF822DD2341F0D130D1F1112309F4BC
:1016800044C00023F1F0B2CF8091C80382FD15C0A1
:10169000112359F0FF2029F08F2D0E9472110E9412
:1016A000261280E00E948409BBCF80E00E94170AC6
:1016B000FF2009F4B5CF8F2DABCF112369F00111B5
:1016C00004C08F2D0E94920AABCF013009F0A8CF41
:1016D0008F2D0E94A911A4CF0111A2CF8F2D0E949E
:1016E000990A8F2D0E94B5118F2D0E94991198CFC4
:1016F000112321F0063008F093CFE3CF053008F036
:101700008FCF8F2D0E94990A8BCF0023D1F3D9332D
:1017100049F43FEF87EE93E0315080409040E1F78D
:1017200000C000008D2F0E94170A7ACF8C2F86955B
:101730008695837069F0813009F072CF8D2F9C2FD0
:101740009370111102C080E090E00E948F2368CF57
:101750008D2F9C2F9370111102C080E090E00E94A9
:101760006A235ECF612F8D2F0E947A0959CF8C2F6B
:101770008370A1F5111154CF4D2F429546954770B6
:10178000440F440F2D2F2F7030E0042E02C0220F83
:10179000331F0A94E2F790E080E0D4FF09C08FE0A5
:1017A00090E002C0880F991F4A95E2F780959095C6
:1017B000C695C695C370822B932BC23049F058F45E
:1017C000C13019F00E944C0D2BCF0E94430D28CF41
:1017D0000E94550D25CF0E94400D22CF86951123E2
:1017E00011F08C2F8170882309F41ACF4D2F429568
:1017F00046954770440F440F2D2F2F7030E0042E74
:1018000002C0220F331F0A94E2F790E080E0D4FF79
:1018100009C08FE090E002C0880F991F4A95E2F757
:1018200080959095C695C695C370822B932BC23038
:1018300049F058F4C13019F00E94B70DF1CE0E9462
:10184000AE0DEECE0E94C00DEBCE0E94640DE8CE30
:10185000CF70112329F08C2F0E947C0D8D2F32CF59
:101860008D2F0E94990A8C2F0E948C0DD9CED23FC9
:1018700041F160F4D03FB9F0D13F81F0112309F478
:1018800043C00111B3CE8C2F8F711FC0D33F01F124
:10189000D43FA1F78091C80382FD24C08C2F8F71A3
:1018A000112311F312C0112341F0053008F0B8CE16
:1018B0008C2F8F710E949E0DB3CE063008F0B0CEF3
:1018C000F7CF8C2F8F711111CFCF0E947C0DA8CE36
:1018D000112329F08C2F8F710E94700DA1CE0E94D0
:1018E0006B0D9ECE112331F063E08C2F8F710E941F
:1018F000381296CE81E00E945612023008F490CE43
:1019000082E00E9456128CCE002359F0D93309F0A0
:1019100009CFEFEFF7EE23E0E150F0402040E1F790
:10192000FFCE8C2F8F71A0CF0F931F93CF93DF9398
:10193000EC01688179818D810E947F0E8C010E946B
:10194000C90D0E943F0DB801CE010E94A00ADF918F
:10195000CF911F910F910895CF93DF93EC018C816C
:10196000882399F0CE010E945008811111C00E9475
:101970006811882351F08D81882339F08091C80344
:1019800082FF03C082E00E945612DF91CF9108953A
:10199000CE010E94940CCE010E940408F6CF882349
:1019A00021F00E9485110E9426120895882321F0BB
:1019B0000E948B110E942612089590E080E00E9400
:1019C0006A2390E080E00E948F230E9492110E947F
:1019D00026120E943C200E94861F08950E94B8246F
:1019E0000E94DD0C08950E9482110E94EE0C089561
:1019F00092959F70963091F058F4925F9F7092305C
:101A000058F4803F19F030F4883E30F481E00895B6
:101A10009A5FF4CF843FD1F380E00895883EB0F31D
:101A2000813FD1F7F3CFFC012481222339F080815B
:101A300091810E94740E0E94F80C089580E0089530
:101A4000A6E0B0E0E6E2FDE00C94F62D2696E2E09A
:101A50000C94122EA7E0B0E0E0E3FDE00C94F62D2C
:101A60002796E2E00C94122E08950E94340D0895FA
:101A70000E94350D9093F1028093F002089508952D
:101A80000E94380D08952091F0023091F102822BCE
:101A9000932B0E94380D08952091F0023091F102AD
:101AA000822393230E94380D08952091F0023091F3
:101AB000F102822793270E94380D08950E94340D69
:101AC00008950E945E0D08950E94610D9093EF02AB
:101AD0008093EE02089590E080E00E94640D0895E6
:101AE00021E030E0A90102C0440F551F8A95E2F7BA
:101AF000CA010E94640D089521E030E002C0220F67
:101B0000331F8A95E2F78091EE029091EF02822BCB
:101B1000932B0E94640D089521E030E002C0220F53
:101B2000331F8A95E2F7209530958091EE029091CF
:101B3000EF02822393230E94640D089521E030E098
:101B400002C0220F331F8A95E2F78091EE02909136
:101B5000EF02822793270E94640D08952091EE02E0
:101B60003091EF02822B932B0E94640D08952091F7
:101B7000EE023091EF02822393230E94640D0895B8
:101B80002091EE023091EF02822793270E94640D8C
:101B900008950895262F277091E001C0990F2A9586
:101BA000EAF723E0769567952A95E1F7660F771FA8
:101BB000660F771FFA01E60FF71F50E040E0682F2D
:101BC00070E08191DF0111979B01042E02C03695D0
:101BD00027950A94E2F721702195282729232827A1
:101BE0002C934F5F5F4F4430510559F70895A82F4C
:101BF000A77023E0969587952A95E1F7880F991F9E
:101C0000880F991FFB01E80FF91F50E040E080E0CA
:101C1000219130E00A2E02C0369527950A94E2F70A
:101C200021703327042E01C0220F0A94EAF7822B79
:101C30004F5F5F4F4430510559F70895262F943078
:101C400070F48B3060F4682F70E08BE0989F600D2B
:101C5000711D112446ED52E0822F0E94CA0D089595
:101C6000292F943068F48B3058F490E066ED72E0E0
:101C70003BE0239F800D911D11240E94F70D0895D4
:101C800080E00895B0E0A0E0E8E4FEE00C94EF2DE1
:101C90007C010091EE021091EF028091F002909190
:101CA000F102082B192BCFE0D0E0CC24C394D12C27
:101CB000BC2EC6010C2E02C0880F991F0A94E2F7B1
:101CC00080239123892B49F4219790F7B12C8B2DF8
:101CD000CDB7DEB7E9E00C940B2EB7018C2F0E9434
:101CE0007715019789F3F3CFCF93DF93EC010E942F
:101CF000420EBE010E947715DF91CF9108951F9388
:101D0000CF93DF93EB019091D502992339F0CB016A
:101D10000E94740EDF91CF911F910895882369F07E
:101D2000CB010E94420E182F682FCE010E941E0E7A
:101D3000BE01812F0E947715EDCFCB010E94300E9E
:101D4000182FF6CF1F93CF93DF93C091F20217E0C5
:101D50008091F3028C1304C0DF91CF911F910895FD
:101D6000D0E01C9FF0011D9FF00D1124EC50FD4FA1
:101D700020813181428153816481758186810E94F5
:101D80002A0D2196C770E4CF20912C0330912D03AA
:101D900040912E0350912F036091300370913103D5
:101DA000809132030E942A0D0895CF93DF93809192
:101DB0003203807F09F04DC080913103882309F4FC
:101DC00048C0E091F2025091F302C0912D03D091EE
:101DD0002C0360912E0370912F0347E05E17C9F129
:101DE0008E2F90E0E49FF0011124EC50FD4F2481F0
:101DF000222391F1489FF001499FF00D1124DF014A
:101E0000AC50BD4F11962C9111972C1325C02C91DD
:101E10002D1322C015962C91159721111DC01296D5
:101E20002D913C91261B370B283C3105A8F480915D
:101E300032038F70806180933203E650FD4F8081C2
:101E40008F70806180838CE293E00E94AC0C0E94D2
:101E5000A20EDF91CF910895FC013196E770BECFBD
:101E6000482F2091F2029091F30257E0291302C00B
:101E700080E0089530E0529FF001539FF00D11244F
:101E8000EC50FD4F8181681306C08081481303C068
:101E900085818111EECF2F5F3F4F2770E7CFA4E1FF
:101EA000B0E0E5E5FFE00C94EC2D8C0186E0F80154
:101EB000DE011F9601900D928A95E1F7F801848169
:101EC000E5809CE2A92E93E0B92E90913003911108
:101ED0001FC08823D1F0EE20A9F0C8010E94130D85
:101EE000F82E882379F087E0F801D50101900D9252
:101EF0008A95E1F7C5010E9471090E94D50E0E94E2
:101F0000C40E5FC0C8010E94AC0CFF24F39459C0FA
:101F1000C080D18082809380F090310320912E0385
:101F200030912F03A401421B530BFF2009F4F9C089
:101F3000483C510508F0A7C0882309F442C090919D
:101F40002D0380913203282F207F09F05CC09D1162
:101F500016C090912C03C91212C0E1104EC08F70B0
:101F60008061809332030E94C40E8CE293E00E9451
:101F7000AC0C80913203F8018683F12C22C0E11071
:101F80003CC06D2D8C2D0E94300F6D2D8C2D0E942C
:101F9000300FE82E8111F1CFCF86D88A8F859889AE
:101FA0000E94740E292F22952F70243078F49F7090
:101FB0002230A8F09923B9F0F8019681907F99F426
:101FC000FE2C8F2D6496ECE00C94082E2A5F2F7067
:101FD000223068F0C8010E94AC0CEF2CF1CF99239D
:101FE00011F0882369F3805E883050F3F3CF803F8F
:101FF00038F3815F833070F7E3CF809132038160E3
:1020000080933203BACF9D1113C090912C03C91253
:102010000FC0E1100DC08683C8010E94AC0C87E0A0
:10202000F801ACE2B3E001900D928A95E1F767CF39
:10203000C8010E94130D882309F464CFEE2009F42F
:1020400061CF80913203803288F020912C0330914F
:102050002D03398728879B868A86909130039C8739
:102060001D868E87CE0108960E94AC0C87E0F80191
:10207000ACE2B3E001900D928A95E1F70E94D50E93
:102080000E94C40E42CF90913203292F207FA1F4E9
:10209000682D9A8A898AA6017A899E2D0E94200D30
:1020A0008CE293E00E94AC0C87E0F50111928A95D6
:1020B000E9F70E94C40E61CF882309F482CF809192
:1020C0002D038D1110C080912C03C8120CC0E1109B
:1020D0000AC09683C8010E94AC0C87E0F5011192FA
:1020E0008A95E9F76ECFC8010E94130D882309F481
:1020F00009CFEE2009F406CF80913203803208F434
:10210000B5CF20912C0330912D033A8329839C82F3
:102110008B82909130039D831E828F83CE01019626
:10212000A3CF483C5105B8F5882309F4EECEFE2C28
:10213000EE2009F4E7CE80912D038D111EC0809111
:102140002C03C8121AC08091320380FD0DC0982F55
:10215000907F51F08683903F09F45ECF982F907F57
:10216000905F8F70892B57CF87E0F801ACE2B3E026
:1021700001900D928A95E1F724CFC8010E94130DBA
:10218000811174CF80913203816080933203C80142
:102190000E94AC0C16CF682D9A8A898AA6017A898A
:1021A0009E2D0E94200D87E0F50111928A95E9F796
:1021B000A6CEAEE0B0E0EFEDF0E10C94F52D28876F
:1021C00039874A875B876C877D878E87CE01089623
:1021D0000E944F0F8823B1F06C85662341F028855B
:1021E00039854A855B857D858E850E942A0D17E09D
:1021F0008091F2029091F30289133DC02E96E3E0A4
:102200000C94112E87E0FE013896DE0111960190A4
:102210000D928A95E1F78C85882349F32091F3028A
:1022200030E0C9010196877099274091F202481762
:10223000190699F097E0929FD001939FB00D112459
:10224000AC50BD4FFE01319601900D929A95E1F789
:102250008093F3020E94A20ECACF0E94F30C109248
:10226000F3021092F20287E0ECE2F3E0DF011D924C
:102270008A95E9F7BCCF819FC00111248C509D4FF6
:102280000E944F0F882309F4B9CFE091F2021E9FFC
:10229000F0011124EC50FD4F2081318142815381A6
:1022A0006481758186810E942A0D8091F20290E0FE
:1022B0000196877099278093F2029ACF80915B03F1
:1022C000869586958695089580915B03877008951D
:1022D00090915B03977081E009F480E0089580910C
:1022E0008703089590918703892B8093870308952E
:1022F0008095909187039823909387030895809306
:102300008703089510928703089590918603892B7F
:1023100080938603089580959091860398239093E7
:102320008603089510928603089508950E949511DA
:10233000089590915C03292F282331F080958923FB
:1023400080935C030E949611089508950E94A51140
:10235000089590915D03292F2823281729F0982BA1
:1023600090935D030E94A611089590915D03292F1B
:10237000282331F08095892380935D030E94A61164
:10238000089580915D03882329F010925D0380E019
:102390000E94A6110895CF93C09187038091860370
:1023A000C82B80915D03882331F0C82B0E94B42391
:1023B00081110E94C1118C2FCF910895CF93DF938B
:1023C000C0910201D09103010E94CB118883C0917A
:1023D0000201D091030148E050E063E573E0CE01D3
:1023E0000E94312E892B59F088E0FE01A3E5B3E06D
:1023F00001900D928A95E1F7CE010E94BC22DF91F7
:10240000CF910895CF93DF93C0910001D091010146
:102410000E94CB118983C0910001D091010140E25B
:1024200050E063E373E0CE010E94312E892B59F016
:1024300080E2FE01A3E3B3E001900D928A95E1F7FB
:10244000CE010E940A23DF91CF9108950E94482572
:10245000813039F48091C70387FF03C00E940212C4
:1024600008950E94DE11089508950E94341208957F
:102470009091C80392FF11C098E0899F90011124A8
:10248000622B60935B030E947C0D80915B038695B9
:10249000869586950E94351208950E947C0D0895B8
:1024A00010925B0380E00E943512089590915B03C7
:1024B0008095892380935B03282F277069F48917FF
:1024C00059F09091C80392FF07C08695869586952E
:1024D0000E948C0D0E9450120895CF93C82F8091B6
:1024E000C80382FB992790F99C17E9F0C0FB82F999
:1024F0008093C8038091C7039091C8030E94CF12B4
:1025000082E00E94561280919A0380FF0CC01F92B5
:10251000CF9387E992E09F938F930E94FB060F90E1
:102520000F900F900F90CF9108958091C80382FB78
:10253000882780F991E089270E946D12089581E033
:102540000E946D12089580E00E946D1208956FEF51
:102550007FEF90E080E00E94832E089590E080E07D
:102560000E944F2E21E0853E9E4F09F020E0822FF1
:10257000089582E090E00E94472E089583E090E065
:102580000E94472E90E00895682F83E090E00E941B
:10259000652E089584E090E00E944F2E0895BC01BE
:1025A00084E090E00E94832E0895AB01BC018FE08F
:1025B00090E00E94772E0895AB01BC0183E190E08A
:1025C0000E94772E089560E070E0CB010E94DC123B
:1025D000089560E070E0CB010E94D5120E94E312E2
:1025E0000895A8E0B0E0E7EFF2E10C94F62D65EE77
:1025F0007EEF90E080E00E94832E60E082E090E039
:102600000E94652E81E090E09093F1028093F002A9
:102610000E94C41260E074E184E090E00E94832E86
:1026200060E086E090E00E94652E60E087E090E048
:102630000E94652E40E050E0BA0188E090E00E94E0
:10264000772E60E083E290E00E94652E60E08CE0EF
:1026500090E00E94652E60E08DE090E00E94652E83
:1026600019821A821B821C821D821E821F8218867A
:1026700048E050E067E170E0CE0101960E94552EDF
:1026800040E050E0BA018FE190E00E94772E0E9476
:10269000E9122896E2E00C94122E0E94F11208959D
:1026A000682F8EE090E00E94652E0895A6E0B0E0CD
:1026B000ECE5F3E10C94F42D0E94F1258C0180915E
:1026C0008803909189038017910781F019821A82FB
:1026D0000E94F125682F49815A81792F80E090E08E
:1026E0000E94410910938903009388032696E4E031
:1026F0000C94102E0E94FD2560939603709397030F
:10270000809398039093990360939203709393033B
:1027100080939403909395030895089508950E94DB
:102720008D13089508950E949213089580E198E210
:102730000E9430180E948E130E948F13089581E02A
:1027400008950E949F1308950E949F13089508956D
:1027500008950E94A7130E94A81308950E94AE1224
:10276000811102C00E944D130E94B91280939A03F6
:102770000E94CA129093C8038093C7030E94BE129E
:102780000E94400D8091EE029091EF020E94610D37
:1027900008950E94E8250E9489170E94AE130E94A6
:1027A0000A090E9493180E9493130895A6E0B0E0CE
:1027B000ECEDF3E10C94EA2D0E94A11381110AC003
:1027C0000E9456130E945E200E9417092696EEE092
:1027D0000C94062E0E949F172AE8822E23E0922E48
:1027E000640110E0F601E190F1906F01812F0E94E9
:1027F00087161F5F143009F44BC0E816F90691F3F1
:1028000080919A0381FD0E9490160E94A413782E55
:1028100010E066246394812F0E9487167C01F401E6
:10282000A190B1904F018A159B0561F100E0CC2485
:10283000C394D12CAE24BF24C5018C219D21892BAA
:10284000C1F07720B1F009831A830E94F1259C839F
:102850008B836D8221E0C7018C219D21892B09F496
:1028600020E049815A816B817C818D81922F0E9469
:1028700041090F5FCC0CDD1C0B30F1F6F4013297EF
:10288000F182E0821F5F143031F60E947A139ACFF2
:10289000E816F90609F0B4CF93CF1F93CF93DF93D7
:1028A0000E947C15EC01C11580E5D807F0F5C11533
:1028B00080E4D80708F09CC0C03ED10520F5CD3C8F
:1028C000D10508F082C0C83AD10578F4C53AD105DF
:1028D00008F073C0C130D10519F1209709F1C43057
:1028E000D105F0F4D0E0C0E01BC0C33CD105D0F767
:1028F000C85AD0E0CC0FDD1FCD5ADE4F0990D881E9
:10290000C02DD4640DC0C11580E2D80708F0D1C035
:10291000C11581E0D80708F05AC0C83ED10510F7AC
:10292000CE01DF91CF911F910895C03682E5D8077F
:1029300018F5C03482E5D80708F06BC0C03282E5D4
:10294000D80708F05FC0C11582E5D80708F497C022
:102950002C2F2695269580E2289F900111248C2FFC
:102960008370C1E0D0E002C0CC0FDD1F8A95E2F792
:10297000C22BD32BDD68D4CFC03A82E5D80760F4F0
:10298000C03882E5D80708F459C0CF71D0E0DC2FF9
:10299000CC27C46FD06AC4CFC03C82E5D80708F406
:1029A00062C0C03E82E5D80708F09CCFDC2FCC2760
:1029B000CC27DF71C06FD06AB3CFC55AD0E0C757FC
:1029C000DE4FC881D0E0D064ABCFD065A9CF8D2FCA
:1029D0000E941E16182FCE0199270E947C15C12F28
:1029E000D0E0DC2FCC27CC27DF71C82BD92B98CF98
:1029F000CE0199270E947C15CC27DF70C82BD92BDC
:102A0000D06A8ECFCF71D0E0DC2FCC27C16FD06AD7
:102A100087CF2C2F26952695277080E2289F90013E
:102A200011248C2F8370C1E0D0E002C0CC0FDD1FD9
:102A30008A95E2F7C22BD32BDC6872CF2C2F269518
:102A40002695277080E2289F900111248C2F837097
:102A5000C1E0D0E002C0CC0FDD1F8A95E2F7C22BA7
:102A6000D32BDA685DCF8C2F8F710E941E16C82F72
:102A7000D0E0DC2FCC27CC27DF71D06251CF8C2F58
:102A80008F710E941E1655E0D695C7955A95E1F7AD
:102A9000CF70D0E0DC2FCC27282F30E084FF05C09A
:102AA00044E0220F331F4A95E1F7C22BD32BD069A4
:102AB00037CF8D2F8F710E941E16182FCE019927A8
:102AC0000E947C15C12FD0E0DC2FCC27CC27DF71F2
:102AD000C82BD92BD2CF462F743030F46B3020F472
:102AE000672F0E942007089590E080E008950E94DB
:102AF0006B150E944D14089582389105B9F1B0F418
:102B00008133910509F47DC048F48932910509F4B7
:102B10006DC08A32910509F47BC008958533910513
:102B200009F45FC08933910509F10895833E910549
:102B3000D9F138F4803E910529F1823E910579F171
:102B40000895863E9105D9F1873E910509F43EC06E
:102B5000843E910541F52091C80321FF24C0809156
:102B6000C70384FD19C087EE90E008952091C70344
:102B7000237009F05AC02091C80323FF14C089E2D2
:102B800090E008952091C70320FD38C03091C8031C
:102B900030FF09C024FF43C090E080E008952091F9
:102BA000C70322FDF7CF08952091C70322FD3AC045
:102BB0003091C80330FD39C024FFF5CFEDCF20910F
:102BC000C70323FFF0CF24FDE7CFCDCF2091C7036C
:102BD00023FD2EC03091C80331FFEECF84EE90E08C
:102BE00008952091C70325FFDECFC9CF2091C703E9
:102BF00025FD21C02091C80323FFD5CF89E390E0B4
:102C0000D2CF2091C70326FFCECF8AE290E008956D
:102C10002091C70326FFC7CF81E390E0089583EE9C
:102C200090E0089582EE90E0089580EE90E008959F
:102C300086EE90E0089585E390E008959091C703B3
:102C400092FF10C041E0282F2471243009F040E0A9
:102C500031E0282F2871283009F030E0431711F0B7
:102C60002CE0822793FF10C041E0282F24712431EB
:102C700009F040E031E0282F2871283109F030E0D8
:102C8000431711F02CE082273091C80330FF10C0A9
:102C900051E0282F2171213009F050E041E0282F28
:102CA0002871283009F040E0541711F029E08227FC
:102CB00031FF10C041E0282F2171213109F040E09F
:102CC00031E0282F2871283109F030E0431711F046
:102CD00029E0822794FD877E0895CF939C01205E92
:102CE0003245C1E02032310538F4FB01C581C11104
:102CF00003C08F710E941C088C2FCF9108950895F6
:102D00000E947F16089508950E9483160895E82F63
:102D1000F0E0EE0FFF1FEF52FC4F8081918108958C
:102D2000B0E0A0E0E6E9F6E10C94EC2D8CEB92E04B
:102D30009F938F930E94FB0681EDE82E83E0F82E8F
:102D40000F900F90912C812C97EBA92E92E0B92E29
:102D500024EBC22E22E0D22E0EEA12E0CCEAD2E020
:102D60009F928F92BF92AF920E94FB06DF92CF920A
:102D70000E94FB06F701819191917F010E94EB086F
:102D80009F938F931F930F930E94FB06DF93CF9324
:102D90000E94FB069FEF891A990AEDB7FEB73C9691
:102DA0000FB6F894FEBF0FBEEDBFF4E08F1691048E
:102DB000B9F6CDB7DEB7ECE00C94082E80EA8A9520
:102DC000F1F7089500C008950E94DE160895F89462
:102DD000E82FE295EF70F0E031A1282F2F7081E00D
:102DE00090E001C0880F2A95EAF7982F90959323D9
:102DF00091A392A1892B82A378940895CF93DF9316
:102E000080E90E94E71681E90E94E71683E90E94A3
:102E1000E71682E90E94E716CCE8D1E089918F3F5E
:102E200011F00E94E71681E0C739D807B9F7DF91A2
:102E3000CF910895AF92BF92DF92EF92FF920F93DE
:102E40001F93CF93DF938C01D62EC62FD0E0CE01F7
:102E500089569E4F7C01FC0120812F3F09F44CC014
:102E6000F894E22FE295EF70F0E031A12F7081E04D
:102E700090E001C0880F2A95EAF7932F982B91A331
:102E800092A18095892382A378940E94E216ECE8AF
:102E9000F1E041E050E0B12CA12C21912F3FB1F1A4
:102EA000A22FA295AF70B0E090968C9190E02F7019
:102EB00002C0959587952A95E2F780FD27C0CA0143
:102EC000A82AB92A440F551F81E0E739F80729F7E6
:102ED000F70180818F3F11F00E94E71661E0A11495
:102EE000B10409F460E08D2D0E94E416CC0FDD1FC3
:102EF000C00FD11FB982A882DF91CF911F910F918E
:102F0000FF90EF90DF90BF90AF90089590E080E049
:102F1000D7CF0E94FE1688E0E1EDF3E0DF01982FA5
:102F20001D929A95E9F7E9ECF3E0DF011D928A958D
:102F3000E9F784E00E94DA170E9480160895A8E05D
:102F4000B0E0E5EAF7E10C94F32D8E010F5F1F4F1F
:102F500088E0F80111928A95E9F7F12C6F2DC801EC
:102F60000E941A17F394F4E0FF12F8CF48E050E003
:102F7000B80189EC93E00E94312E21E0009709F41A
:102F800020E0892B41F088E0F801A9ECB3E0019042
:102F90000D928A95E1F744E061ED73E089EC93E0EE
:102FA0000E94DB17182F0E948416812F2896E5E0D7
:102FB0000C940F2E0895B0E0A0E0E1EEF7E10C9440
:102FC000F02D6C017B01042FC22F222379F081E0C8
:102FD00080939D030E94F12590939C0380939B0313
:102FE00080E0CDB7DEB7E8E00C940C2ED0919D03C5
:102FF000DD23B1F380919B0390919C030E940926ED
:10300000059770F310E0000F111FA801B601C7016A
:103010000E94312E892B31F0A801B601C7010E9410
:103020003E2ECD2F10929D038C2FDBCF0E94D61306
:1030300008950E948A250E9472280E9496130E9479
:103040008C280E94C9130E9499280E949E280E94E1
:1030500016180E94C4280E94A7260E94A913F5CF23
:103060009093CF028093CE020895FB012581222305
:1030700041F097FF06C09F77BC0190E080E00E947E
:103080009D1981E008950F931F93CF93DF93EC0177
:103090008B01FB018581882389F00E946F11827268
:1030A000FE01E053FC47E830F10540F4E955F14DED
:1030B0000C94E02D882369F00E94CF18B801CE014E
:1030C0000E943518DF91CF911F910F9108958823A9
:1030D00099F30E94CE18F2CF80E00E94AE18EECF96
:1030E00081E0FBCF82E0F9CF83E0F7CF84E0F5CF3A
:1030F00085E0F3CF9091DA03923071F48A3050F486
:1031000090E009966AE070E00E94CC2D875A0E94F8
:10311000890A08958650FBCF0E94F42108950895EE
:103120000E948F1808958CE090E00E94472E8093B3
:10313000DA030E94901880919A0380FF0EC080915C
:10314000DA031F928F9382EF92E09F938F930E94F6
:10315000FB060F900F900F900F900895CF93C82FFC
:103160008093DA03682F8CE090E00E94652E8C2F0C
:103170000E94901880919A0380FF0EC08091DA031C
:103180001F928F9383ED92E09F938F930E94FB0693
:103190000F900F900F900F90CF910895089508957C
:1031A0000E94B9228093D9039091DA03913029F4D7
:1031B00081FF03C089E30E94890A0E946F118093F6
:1031C000DB030E9482110E9492118091DA03823007
:1031D00021F158F48823C1F08130D1F08FE39CE9CC
:1031E0000197F1F700C000000895843051F1853057
:1031F000A9F78BE191E00E94A40785E290E00E948C
:10320000A40788E290E006C082EE0E948409E6CF1F
:1032100088E193E00E94A407E1CF8091D90380FD6B
:1032200003C083E50E94890A82EE0E9484098FE32D
:103230009CE90197F1F700C0000087E50E94890A28
:10324000CDCF86EE0E94890A88E1F8CF8091DA031B
:10325000823011F148F4882381F0813091F080911F
:10326000DB030E947F1108958430F9F08530B9F7AF
:1032700088E290E00E94A407F2CF82EE0E94170A33
:10328000EECF8CE20E94890A8091D90381FFE7CFBB
:1032900089E30E94890AE3CF82EE0E94170A809197
:1032A000D90380FDDCCF83E5F4CF88E2F2CF8F92A3
:1032B0009F92AF92BF92EF92FF920F931F93CF9383
:1032C000DF934B015C01D091DA038CE1E82EF12C05
:1032D00007E010E021E0D501C4010E2C04C0B69532
:1032E000A795979587950A94D2F7C82FCF70222378
:1032F00039F0D43051F4CA3040F080E00E947A189E
:103300008C2F0E947A1820E005C0C111F9CF04303B
:103310001105B4F30150110984E0E81AF1080F3FD8
:103320001007C9F6DF91CF911F910F91FF90EF9099
:10333000BF90AF909F908F900895CF92DF92EF92C1
:10334000FF926B017C01C114D10481E1E806F10414
:10335000A0F5C114D10481E0E806F10420F08091C9
:10336000DA03823051F10E94D018C114D10481E0F7
:10337000E806F10438F18091DA03811123C081E07D
:10338000E81AF108C701B6012AE096958795779566
:1033900067952A95D1F778528F4F9F4F0E94571902
:1033A00083E0D822EE24FF24C701B60174528F4F68
:1033B0009F4F0E9457190E942619FF90EF90DF90AF
:1033C000CF900895C701B601F4CF809104011F92F8
:1033D0008F93809105011F928F93809108011F9216
:1033E0008F93809109011F928F9380910A011F9200
:1033F0008F9380910B011F928F9382E193E09F93B3
:103400008F930E94FB068DB79EB70E960FB6F89469
:103410009EBF0FBE8DBF0895883248F58E3108F0EB
:103420007FC08B3069F130F4873009F4E0C081E768
:1034300094E0F1C0833109F468C08431C1F783E9B5
:1034400094E09F938F930E94FB060F900F908091C2
:10345000A203882309F411C11092A2031092A103C0
:103460001092A00310929F0310929E0325C08F34E8
:1034700009F4D6C008F03FC0893209F38833B9F6A1
:1034800086E994E09F938F930E94FB060E94E519C2
:103490001F9281E08F931F9288E08F938FE893E0D3
:1034A0009F938F930E94FB068DB79EB708960FB629
:1034B000F8949EBF0FBE8DBF2091A203222309F472
:1034C000D3C080919E0390919F03009711F48BE9E4
:1034D00091E09F938F931F922F938FE594E09F939A
:1034E0008F930E94FB060F900F900F900F900F90FC
:1034F0000F9081E00895813509F4A6C008F4A6C0B4
:10350000823509F094CF81E08CC085E894E09F93E8
:103510008F930E94FB060E94E5190F900F90CCCF6D
:103520008D518093A203833009F446C078F4813032
:10353000E1F08230C1F11092A20382E894E09F93FF
:103540008F930E94FB060F900F901BC0853009F4EB
:1035500045C0D8F1863079F784E091E09093A103DB
:103560008093A00383EE91E008C08BE091E09093FC
:10357000A1038093A0038FE991E090939F03809330
:103580009E038091A203882309F496CF1F928F9304
:103590008EE794E09F938F930E94FB060F900F900D
:1035A0000F900F9089CF8AE091E09093A1038093D0
:1035B000A00388EA91E0E1CF89E091E09093A10334
:1035C0008093A00384EB91E0D8CF88E091E09093C2
:1035D000A1038093A00381EC91E0CFCF85E091E03F
:1035E0009093A1038093A00380ED91E0C6CF81E08A
:1035F00080930B0184E180930A018AE080930901A2
:103600008EE18093080188E08093050188E2809331
:10361000040184E794E09F938F930E94FB067DCF83
:103620008AE0E091A003F091A1033097D1F02081CE
:10363000082E000C990B820F911D8F3F910541F0D0
:103640003CF08FEF808307C08FEFEBCF86EFE9CFA1
:1036500097FFF8CF108280811F928F938BE694E0C2
:1036600099CF88E694E0D7CF8BE594E09F938F9332
:103670000E94FB060F900F903CCF80E00895CF93FF
:10368000C82F1F928F938CEA94E09F938F930E9490
:10369000FB0681E090E002C0880F991FCA95E2F70F
:1036A0000E94400D0E94F30C0F900F900F900F900E
:1036B000CF910895B0E0A0E0E0E6FBE10C94F12D9D
:1036C000EBEFE80FEF3308F054C1F0E0E155F14DB6
:1036D0000C94E02D0E94BE129F938F938CE598E08E
:1036E0009F938F930E94FB060E94B91283FB992738
:1036F00090F91F929F9382FB992790F91F929F93B5
:1037000081FB992790F91F929F93982F91701F9298
:103710009F931F928F9383E198E09F938F930E94D2
:10372000FB060E94CA1293FB222720F91F922F93B7
:1037300087FB222720F91F922F9386FB222720F94F
:103740001F922F9385FB222720F91F922F9384FB32
:10375000222720F91F922F9383FB222720F91F9203
:103760002F9382FB222720F91F922F9391FB222770
:1037700020F91F922F93292F21701F922F9381FBE5
:10378000222720F91F922F93282F21701F922F9309
:103790009F938F9384E197E09F938F930E94FB0602
:1037A0008DB79EB78A960FB6F8949EBF0FBE8DBF99
:1037B00081E02AC08CE199E09F938F930E94FB06E1
:1037C0000E944D130F900F90F3CF8FE595E09F93DC
:1037D0008F930E94FB06F6CF80919A03807F80939F
:1037E0009A0388E395E09F938F930E94FB0688E1FC
:1037F00099E09F938F930E94FB0681E08093A3033F
:103800000F900F900F900F90CDB7DEB7E7E00C94BC
:103810000D2E8CEF98E09F938F930E94FB060E94E1
:103820004408D0CF90919A03892F8E7F90FF8160BA
:1038300080939A0380FF03C080EF98E0C8CF83EEA7
:1038400098E09F938F930E94FB0680919A03817F5B
:1038500080939A03B7CF90919A03892F8D7F91FF20
:10386000826080939A0381FF0AC086ED98E09F935F
:103870008F930E94FB0680919A038160E9CF88ECC8
:1038800098E0A5CF90919A03892F8B7F92FF846057
:1038900080939A0382FF03C089EB98E0E8CF89EA1E
:1038A00098E095CF90919A03892F877F93FF886046
:1038B00080939A0383FF03C08DE998E0D8CF80E915
:1038C00098E085CF88EF91E09F938F9385E395E013
:1038D0009F938F930E94FB060F900F900F900F9075
:1038E00067CF0E94FD25062FF72EE82ED92EC09116
:1038F000C703C7FBCC27C0F90E946825182F0E9478
:103900004825D82F0E94AC22DF92EF92FF920F93AE
:103910001F92CF931F921F931F92DF931F928F933B
:1039200081EB94E09F938F930E94FB068DB79EB727
:103930000E960FB6F8949EBF0FBE8DBF39CF0E9472
:10394000F30C9091C703892F97FB87F980588093D8
:10395000C70387FF03C086E898E039CF8BE798E07C
:1039600036CF80E00E943F1B23CF8953FBCF8D5180
:10397000F9CF89E798E09F938F930E94FB060F9001
:103980000F9080E041CF80E008950E94C31C08950D
:10399000CF93C82F8091A3038130C1F0882339F0E1
:1039A000823009F450C01092A30380E00DC00E9441
:1039B0006F118232D1F78C2F0E94C31C81111FC05E
:1039C0008C2F0E945A1B8170CF9108950E946F1115
:1039D000823289F38C2F0E94C51C811127C0C4310B
:1039E00039F180F4CB3091F0C03131F186EA94E0C6
:1039F0009F938F930E94FB060F900F901BC081E056
:103A000090E0E1CFC932A1F0C83381F788E395E0B7
:103A10009F938F930E94FB0688EA94E09F938F9375
:103A20000E94FB060F900F900F900F9081E0CBCF7C
:103A30001092A30380E0C7CF82E08093A30388E3C2
:103A40000E940C1AF3CF8C2F0E940C1A81E0BCCF7D
:103A5000CF93DF93EB0186319C4711F50E946F11E4
:103A60009D81992399F08A7A91E009F490E09093EE
:103A7000A403811109C089E20E9484240E942612B5
:103A800080E0DF91CF91089585E3F6CF8091A40384
:103A9000811104C089E20E949E24F0CF85E3FBCF10
:103AA00081E0EFCFCF93DF93EC01FB018581882389
:103AB00009F4D2C09E0130572332310508F0B2C05C
:103AC0000E94CA129093C8038093C703FE01E1507D
:103AD000F047E232F10520F4E251F14D0C94E02D73
:103AE0008091C70381608093C70393C08091C8030E
:103AF00088608093C8038DC08091C7038260F3CF34
:103B00008091C7038460EFCF8091C7038860EBCFBB
:103B10008091C8038160EDCF8091C8038260E9CFB6
:103B20008091C7038061DFCF8091C7038062DBCFC4
:103B30008091C7038064D7CF0E94F30C8091C703A4
:103B40008068D1CF8091C7038C60CDCF8091C803AE
:103B50008360CFCF8091C7038E7FC5CF8091C8038C
:103B6000877FC7CF8091C7038D7FBDCF8091C7036B
:103B70008B7FB9CF8091C703877FB5CF8091C80372
:103B80008E7FB7CF8091C8038D7FB3CF8091C7035D
:103B90008F7EA9CF8091C7038F7DA5CF8091C7036A
:103BA0008F7BA1CF0E94F30C8091C7038F779BCFAF
:103BB0008091C703837F97CF8091C8038C7F99CF73
:103BC0008091C70382FB992790F921E0922790FB0F
:103BD00082F990FB83F987CF8091C803982F909545
:103BE00091708E7F892B90FB81F983CF9091C703D1
:103BF000892F8F7B96FF806476CF0E94F30C909183
:103C0000C703892F97FB87F980586DCF81E00E9409
:103C100050138091C7039091C8030E94CF120E9455
:103C2000F30C80E0DF91CF91089580E0F0CF909188
:103C3000C703892F8F7E94FF806155CF9091C70372
:103C4000892F8E7F90FF81604ECF9091C803892F7E
:103C5000877F93FF88604DCF81E0E4CF282F35EB3D
:103C60002303C001112497FF04C080589109892FB4
:103C7000089580589F4FFBCF8091AB0380FF0DC00C
:103C80006091090170E0660F771F6038710570F56B
:103C90006115710569F1862F089581FF07C0609154
:103CA000090184E0689FB0011124EFCF6091090100
:103CB00082FD0AC08091AA038823A9F020910801FF
:103CC00060910901821710F088E0ECCF869FC00157
:103CD000112433E0880F991F3A95E1F7622F70E0C5
:103CE0000E94CC2DD2CF68E070E0D5CF8FE7089549
:103CF00081E008958091AB0380FF0CC060910501C5
:103D000070E075956795759567956115710549F131
:103D1000862F089581FF06C06091050170E07595BA
:103D20006795F3CF6091050182FD0BC09091A903C7
:103D30009923A1F06091040180910501961738F054
:103D4000682F70E06038710500F38FE70895899F50
:103D5000C001112470E00E94CC2DF4CF61E070E02E
:103D6000D7CF81E008958D3C31F40E943C1E8195AF
:103D70008093AF0308958E3C19F40E943C1EF8CF47
:103D80008F3C31F40E943C1E81958093AE030895D0
:103D9000803D19F40E943C1EF8CF893D29F40E9411
:103DA0007A1E8093B00308958A3D21F40E947A1E02
:103DB0008195F7CF8B3D31F40E947A1E81958093D7
:103DC000B10308958C3D19F40E947A1EF8CF9FE24A
:103DD000980F983070F4815D990B21E030E001C0BC
:103DE000220F8A95EAF78091AD03822B8093AD0371
:103DF00008958D3D31F48091AB0381608093AB03D6
:103E000008958E3D21F48091AB038260F7CF8F3D02
:103E1000B9F78091AB038460F1CF4091AE038D3C44
:103E200059F48091AF0387FF0DC01092AF03411189
:103E30000BC01092AA0308C08E3C81F48091AF039E
:103E400018169CF3442381F08091B0039091B10344
:103E5000892B09F05AC01092A90308958F3C49F4A8
:103E600047FFF0CF1092AE038091AF038111ECCFEA
:103E7000E0CF803D19F41416ACF3E4CF9091B00379
:103E8000893D29F41916F4F61092B003DBCF8A3D70
:103E900019F497FFD7CFF8CF9091B1038B3D29F458
:103EA00097FFD0CF1092B103CDCF8C3D19F41916E6
:103EB000CCF3C8CF9FE2980F983090F4815D990BB6
:103EC00021E030E0B90102C0660F771F8A95E2F762
:103ED000CB0180959091AD0389238093AD03B2CF40
:103EE0008D3D31F48091AB038E7F8093AB03AACFDD
:103EF0008E3D21F48091AB038D7FF7CF8F3D09F08C
:103F0000A1CF8091AB038B7FF0CF089580919A036E
:103F100083FF96C084E599E09F938F930E94FB06F0
:103F20008091AD031F928F938FE499E09F938F93BD
:103F30000E94FB068DE499E09F938F930E94FB06FD
:103F40008091AE03282F082E000C330B3F938F93E4
:103F50008AE499E09F938F930E94FB0688E499E09E
:103F60009F938F930E94FB068091AF03282F082E0A
:103F7000000C330B3F938F9385E499E09F938F93CD
:103F80000E94FB0683E499E09F938F930E94FB06B7
:103F90008091B003282F082E000C330B3F938F9392
:103FA00080E499E09F938F930E94FB068EE399E053
:103FB0009F938F930E94FB068091B103282F082EB8
:103FC000000C330B3F938F938BE399E09F938F9378
:103FD0000E94FB0688E399E09F938F930E94FB0663
:103FE0008DB79EB780960FB6F8949EBF0FBE8DBF5B
:103FF0008091AA031F928F9385E399E09F938F93FB
:104000000E94FB0683E399E09F938F930E94FB0637
:104010008091AB031F928F9380E399E09F938F93DE
:104020000E94FB068DE299E09F938F930E94FB060E
:104030008DB79EB70C960FB6F8949EBF0FBE8DBF7E
:104040000E94F1259C019091AE038091AF03982BC3
:1040500021F03093A8032093A7039091B00380919F
:10406000B103982B21F03093A6032093A5038CEA8B
:1040700093E00E945C23089586E0ECEAF3E0DF0120
:104080001D928A95E9F71092AA031092A903109243
:10409000AB030895FC01828181110EC083818111DF
:1040A0000BC08481811108C091E08581811101C01C
:1040B00090E0892F8170089581E0FCCFA6E0B0E008
:1040C000E4E6F0E20C94F52D86E0ECEAF3E0DE01A4
:1040D000119601900D928A95E1F71092AE0310921D
:1040E000AF031092B0031092B1038B819C81892B96
:1040F00089F08091A7039091A8030E940926AC0142
:104100009091AA039923C9F180910A018417150699
:1041100008F440C08D819E81892B91F08091A50388
:104120009091A6030E940926AC019091A9039923BE
:1041300009F46AC0809106018417150608F472C05C
:10414000BE016F5F7F4F8CEA93E00E94D224811101
:1041500005C08CEA93E00E944A2081110E94861FCC
:1041600086E0FE013196ACEAB3E001900D928A95AB
:10417000E1F72696E3E00C94112E20910B018AE0E2
:10418000289F900111242417350720F69F5F9093F4
:10419000AA0302C09F3FD1F71B81112359F00E944F
:1041A0003C1E9FEF11160CF491E0899F802D112485
:1041B0008093AE031C81112359F00E943C1E9FEF97
:1041C00011160CF491E0899F802D11248093AF0388
:1041D0008091AE03882309F49DCF1091AF03112382
:1041E00009F498CF0E942E1E882351F08093AE03CD
:1041F000812F0E942E1E882329F08093AF038ACF3F
:1042000081E0F4CF81E0F9CF209107018AE0289F77
:10421000900111242417350708F092CF9F5F9093E7
:10422000A90302C09F3FD1F71D81112359F00E94BD
:104230007A1E9FEF11160CF491E0899F802D1124B6
:104240008093B0031E81112359F00E947A1E9FEFC4
:1042500011160CF491E0899F802D11248093B103F5
:104260008091B003882309F46BCF1091B10311231F
:1042700009F466CF0E942E1E882351F08093B0036C
:10428000812F0E942E1E882329F08093B10358CFDE
:1042900081E0F4CF81E0F9CFB0E0A0E0E2E5F1E227
:1042A0000C94EF2DE82FF0E0E958F64FB490282F4A
:1042B00026952695269530E0F901E95EF54F0491A3
:1042C000877010E0082E02C0159507950A94E2F752
:1042D00001701127F901E95FF54FE490F12C082EE8
:1042E00002C0F594E7940A94E2F791E0E922FF24F2
:1042F000F901E950F64FC491D0E002C0D595C795B9
:104300008A95E2F7C170DD27C62ED12C0115110563
:1043100049F5E114F10431F086EE0E948409C601EA
:10432000009771F5B6018B2D0E94710AC6010097A6
:1043300079F5E114F104A1F50115110531F081EED3
:104340000E94170AC6010097C9F5CD2B31F08CE207
:104350000E94890AC114D104C9F5CDB7DEB7E9E0DE
:104360000C940B2E81EE0E948409C601009789F2FD
:10437000EFE9FFE03197F1F700C000000197F6CFB9
:10438000EFE9FFE03197F1F700C000000197C8CFD7
:10439000EFE9FFE03197F1F700C000000197C7CFC8
:1043A00086EE0E94170AC601009731F2EFE9FFE09E
:1043B0003197F1F700C000000197F6CFEFE9FFE079
:1043C0003197F1F700C000000197BDCF8FE99FE062
:1043D0000197F1F700C0000091E0C91AD108BACFE7
:1043E00060E00E944C210895982F9F709A5096305B
:1043F00020F0805D0E94F0210895895AFBCF0F9331
:104400001F93CF93DF93C42FD22FFC018581882384
:10441000C9F04093B4030E94F1259093B3038093B5
:10442000B20380E28C0F883040F4C77081E001C095
:10443000880FCA95EAF70E94920ADF91CF911F91E7
:104440000F9108951091B403141332C08091B203F8
:104450009091B3030E940926883C910548F5C0E27B
:10446000CD0F1D17B9F080E2810F883040F417702E
:1044700081E001C0880F1A95EAF70E94990AC830B6
:1044800048F481E09D2F977001C0880F9A95EAF754
:104490000E94920A802F0E94890AC83070F6D77055
:1044A00081E001C0880FDA95EAF70E94990AC5CF2A
:1044B00080E28C0F883008F6C77081E001C0880F59
:1044C000CA95EAF7F2CF0F93DB0188519C478730FA
:1044D0009105A0F5FC01E05FF04D0C94E02D06E2A3
:1044E00021EE41EE6AE17CE7CD010E94FF2180E0F0
:1044F0000F91089507E225EE45EE6BE17CE7F4CFDE
:1045000006E221EE40EE68E17CE7EECF07E225EE21
:1045100044EE69E17CE7E8CF06E221EE42EE6CE191
:104520007CE7E2CF07E225EE46EE6DE17CE7DCCFEB
:1045300008E221E045EE6EE17CE7D6CF15968C913E
:10454000882319F01092B403D3CF81E0D1CF909398
:10455000BA038093B9030895E091B903F091BA03C7
:10456000309729F00190F081E02D0995089580E0C1
:1045700008950E94AC220895EF92FF920F931F932B
:10458000CF93DF93EC01E091B903F091BA03309738
:10459000E1F10280F381E02D099580919A0382FF79
:1045A00034C080FF0DC088811F928F938CE49AE005
:1045B0009F938F930E94FB060F900F900F900F9088
:1045C0007E0186E0E80EF11C06E41AE080919A0371
:1045D00080FF0BC08A811F928F931F930F930E94BD
:1045E000FB060F900F900F900F902196CE15DF05D0
:1045F00069F780919A0380FF08C084E49AE09F9352
:104600008F930E94FB060F900F90CDB7DEB7E6E0C8
:104610000C940E2EEF92FF920F931F93CF93DF9384
:10462000EC01E091B903F091BA03309709F43FC06F
:1046300086E088830480F581E02DCE010995809184
:104640009A0382FF34C080FF0DC089811F928F932F
:104650008FE29AE09F938F930E94FB060F900F903A
:104660000F900F907E018EE1E80EF11C09E21AE036
:1046700080919A0380FF0BC08A811F928F931F93B2
:104680000F930E94FB060F900F900F900F902196B2
:10469000CE15DF0569F780919A0380FF08C087E295
:1046A0009AE09F938F930E94FB060F900F90CDB7D7
:1046B000DEB7E6E00C940E2EE091B903F091BA0358
:1046C000309739F022E0DC012C930680F781E02D51
:1046D00009950895A3E0B0E0E0E7F3E20C94F62D2D
:1046E0002091B7033091B80328173907A1F09093B0
:1046F000B8038093B703E091B903F091BA03309700
:1047000051F023E029839B838A830084F185E02D87
:10471000CE01019609952396E2E00C94122EA3E0B7
:10472000B0E0E5E9F3E20C94F62D2091B503309169
:10473000B60328173907A1F09093B6038093B50309
:10474000E091B903F091BA03309751F024E0298346
:104750009B838A830084F185E02DCE010196099523
:104760002396E2E00C94122ECF93DF93C0910201C6
:10477000D091030122960E944825813081F48091D6
:10478000C70387FF0CC0C0910001D09101012296A0
:104790009EE180E0915028F4DF91CF91089596E05A
:1047A000F8CF29912223B1F38F5FF4CFCF93C82F95
:1047B000811102C080E024C00E944825813011F59B
:1047C0008091C70387FF1EC0EC2FE695E695E6951E
:1047D000EE3180F78091000190910101E80FF92FEF
:1047E000F11D228130E0C77081E090E002C0880FA7
:1047F000991FCA95E2F72823392381E0232BD1F2B0
:10480000CF9108958091020190910301FC013296AD
:10481000089621912C1721F0E817F907D1F7CACF94
:1048200081E0EECF9C01FC0132969FEF80E0419148
:10483000461751F09F3F19F4411101C0982F8F5F27
:104840008630A9F79F3F09F40895290F311D97FD80
:104850003A95F90162830895FC01329608962191F8
:10486000261303C0DF0111971C92E817F907B9F767
:104870000895E62FE695E695E695EE3170F4E80F9B
:10488000F92FF11D677021E030E001C0220F6A9519
:10489000EAF78281822B8283089580919A0380FFB8
:1048A0000CC01F926F9383E89AE09F938F930E94AE
:1048B000FB060F900F900F900F900895E62FE6954E
:1048C000E695E695EE3178F4E80FF92FF11D677063
:1048D00021E030E001C0220F6A95EAF7209582813D
:1048E00028232283089580919A0380FF0CC01F9291
:1048F0006F9385E69AE09F938F930E94FB060F903B
:104900000F900F900F900895CF93C82F0E944825C5
:104910006C2F813061F48091C70387FF08C08091BC
:104920000001909101010E943924CF910895809156
:104930000201909103010E941224F7CFCF93C82F58
:104940000E9448256C2F813061F48091C70387FF56
:1049500008C080910001909101010E945E24CF91D6
:10496000089580910201909103010E942C24F7CFB9
:104970000E944825813079F48091C70387FF0BC0DE
:10498000E0910001F091010132968EE1DF011D926C
:104990008A95E9F70895E0910201F09103013296BA
:1049A00086E0F4CFDC01FB0111969C911197818187
:1049B000981322C012968C911297882319F0928135
:1049C00089131AC013968C911397882319F0938139
:1049D000891312C015968C911597882319F095812B
:1049E00089130AC014969C91992321F081E02481B7
:1049F000291303C080E001C081E08170089508950B
:104A00000E94FF24089581110EC081E080930F0160
:104A100060910C0170910D0180910E0190910F0138
:104A20000E940025089582E0F1CF83E080930F017A
:104A300060910C0170910D0180910E0190910F0118
:104A40000E94002508950E940325089581E0809327
:104A50000F0160910C0170910D0180910E019091F8
:104A60000F010E94002508950E942625089591E0D7
:104A7000811101C090E090930E0160910C01709142
:104A80000D0180910E0190910F010E940025089563
:104A900080910E01089580930D0160910C01709139
:104AA0000D0180910E0190910F010E940025089543
:104AB00080910D01089580930C0160910C0170911B
:104AC0000D0180910E0190910F010E940025089523
:104AD00080910C010895089508950E946C25089511
:104AE000089508950E946B250895CF930E94702524
:104AF0000E949F170E947125C0E08C2F0E9487168C
:104B0000892B31F4CF5FC430C1F780E0CF91089595
:104B100081E0FCCF85B7806885BF85B7806885BF99
:104B200008951F921FB61F9211248F939F93AF93E6
:104B3000BF938091BB03811113C08091DC039091DE
:104B4000DD03A091DE03B091DF034196A11DB11DED
:104B50008093DC039093DD03A093DE03B093DF0327
:104B6000BF91AF919F918F911F901FBE1F9018957D
:104B70008091E403843031F10E94C9081092BB0394
:104B800088E190E020E40FB6F894A8958093600047
:104B90000FBE2093600083B7817F846083BF83B79B
:104BA000816083BF7894889583B78E7F83BF0FB66B
:104BB000F894A895809160008861809360001092BD
:104BC00060000FBE08950E94F30C0E94CE08089565
:104BD00082E084BD93E095BD9AEF97BD80936E000F
:104BE00008952FB7F8948091DC039091DD03A09194
:104BF000DE03B091DF032FBF08952FB7F8946091C3
:104C0000DC037091DD038091DE039091DF032FBF01
:104C100008959C014FB7F8948091DC039091DD03D7
:104C2000A091DE03B091DF034FBF821B930B089569
:104C300078941F921FB61F9211248F939F93AF9366
:104C4000BF938091DC039091DD03A091DE03B091CE
:104C5000DF030196A11DB11D8093DC039093DD035A
:104C6000A093DE03B093DF03BF91AF919F918F912B
:104C70001F901FBE1F90189587E797E79093010834
:104C80008093000888E19AE00FB6F894A895809385
:104C900060000FBE90936000FFCF88E19AE00FB6EE
:104CA000F894A895809360000FBE90936000FFCFAA
:104CB0009B01BA019091E4039430E9F48F708093E2
:104CC000E9009FEF8091E800915085FD06C085EDD9
:104CD0008A95F1F700009111F5CF8091E80085FFEA
:104CE0000AC050E040E0C9010E943A298091E800E2
:104CF0008E778093E800089543E050E0BC0182E0A5
:104D00000E945826089546E050E0BC0182E00E94CF
:104D10005826089540E250E0BC0182E00E945826E7
:104D20000895CF93DF93EC010E94482548E050E0BE
:104D3000BE0181E00E94582688E0FE01AFEBB3E09F
:104D400001900D928A95E1F7DF91CF910895089532
:104D500087EC9AE09F938F930E94FB068091E30378
:104D60000F900F90811109C00E94CA2A0E94272B20
:104D70008091E20084608093E200089583EC9AE0E1
:104D80009F938F930E94FB061092E3030F900F9066
:104D900008958FEB9AE09F938F930E94FB060E94E9
:104DA000262581E00E9437250F900F9008958BEB08
:104DB0009AE09F938F930E94FB066091E00381E04D
:104DC000611101C080E00E9415250F900F90089599
:104DD00087EB9AE09F938F930E94FB069091E403E8
:104DE00081E0943009F080E06091E0030E94232587
:104DF0000F900F9008952091BD032F5F822F62E3E3
:104E00000E94C02D992319F02093BD03089510929C
:104E1000BD038091BE038823F1F08091E4038430C8
:104E2000C1F49091E9009F702091EC00822F817075
:104E300020FD80E8892B93E09093E9009091EB00AE
:104E400090FF04C09091EE0097FD08C08F70809392
:104E5000E9001092BE0308951092F1009091E800CD
:104E600095FDFACF9091E80090FFF0CF9091E80087
:104E70009E779093E800EACF42E061EC81E00E94E7
:104E8000462A42E261EC82E00E94462A42E261EC5C
:104E900083E00E94462A9091E40381E0943009F077
:104EA00080E06091E0030E94032508958091E6036D
:104EB000833009F461C030F48130D1F1823009F4DB
:104EC0009EC008958A3009F48AC08B3009F46FC0FF
:104ED000893009F050C08091E503813209F04BC060
:104EE0008091E9039091EA03029708F044C0809111
:104EF000E800877F8093E8008091E80082FF37C058
:104F00009091F3008091F200029731F48091F100CA
:104F1000813011F0863021F48091F1000E944B2500
:104F20008091E8008B778093E8000E947A2A23C062
:104F30008091E503813AF9F48091E800877F8093BE
:104F4000E8008091E9039091EA03892B61F468E01D
:104F50008FEB93E070E00E9489298091E8008B77C5
:104F60008093E800089560E090E080E0F3CF8091C6
:104F7000E4038111C1CF08958091E503813AD9F707
:104F80008091E9039091EA03892BA9F78091E800C9
:104F9000877F8093E8008091E80080FFFCCF0E942B
:104FA00048258093F1008091E8008E77BCCF8091F6
:104FB000E503813201F78091E9039091EA03892B9F
:104FC000D1F68091E800877F8093E8000E947A2ADA
:104FD0008091E7030E9437250E94F30C0895809189
:104FE000E503813241F68091E800877F8093E800F5
:104FF0000E947A2A8091E8030E945B25089580919F
:10500000E503813A09F0B7CF8091E800877F80936C
:10501000E8008091E80080FFFCCF0E946825C1CFA6
:105020009FB7F8941092BE039FBF9091E403943011
:1050300009F048C02091E9002F703091EC00932FC7
:10504000917030FD90E8922B23E02093E9002091AD
:10505000EB0020FF34C02091EE0027FF30C02091EC
:10506000BC03222321F02091E80025FF28C01092E4
:10507000BC0326E03091E80035FF14C08093F100B6
:105080008091E80085FD27C08091E80080FFFCCF7B
:105090008091E8008E778093E8009F709093E900FC
:1050A00080E008953091E403343049F43091EB000E
:1050B00035FD05C0215041F481E08093BC039F7011
:1050C0009093E9008FEF0895EFE9FFE03197F1F752
:1050D00000C00000CFCF8FB7F89421E02093BE032B
:1050E0008FBFDBCF84B7877F84BF0FB6F894A895B6
:1050F00080916000886180936000109260000FBE14
:1051000080E890E00FB6F89480936100909361007E
:105110000FBE0E94342508950E94CA2A0E94272BA0
:10512000E2EEF0E080818460808378940E94A52D77
:10513000089580E191E00E94A72208958091E40300
:10514000853091F480919A0380FF08C081EA9AE04B
:105150009F938F930E94FB060F900F908091E40322
:10516000853019F00E94E32508950E94B8250E9419
:105170007525882399F38091E203882379F30E94AF
:1051800024290E94F30CEACF08959A014091EB0381
:105190005091EC030E94CD280895492F55274330A4
:1051A000510521F168F44130510509F443C0423002
:1051B000510509F444C090E080E050E040E026C092
:1051C0004132510551F142325105A9F76330710561
:1051D00090F7FB01EE0FFF1FEF53FD4F4081518110
:1051E00062547D4FFB01808190E010C0992781308F
:1051F000910581F0009729F00297E9F6EBECFAE0CF
:1052000002C0E5EFFAE0849190E0AF01F90151832B
:1052100040830895EBEDFAE0F6CF6330710558F660
:10522000660F771FFB01E953FD4F4081518189E0F3
:1052300090E0ECCF82E190E04DE45BE0E7CF84E5E5
:1052400090E049EF5AE0E2CF80E189BD82E189BD7B
:1052500009B400FEFDCF8091D8008F7D8093D800E7
:105260008091E00082608093E0008091E00081FD09
:10527000FCCF0895AF92BF92CF92DF92FF920F932F
:105280001F93CF93DF936C01EB018A010E94992A4F
:10529000F82E811123C00115110539F0F801808124
:1052A0009181C81BD90BC80ED91EB12CA12C2097F7
:1052B000A9F08091E80085FD22C08091E8008E77FA
:1052C0008093E80001151105A1F0F801808191811A
:1052D000A80EB91EB182A08285E0F82E8F2DDF9135
:1052E000CF911F910F91FF90DF90CF90BF90AF9023
:1052F00008950E94992A8823D1F2F82EEFCFF60163
:1053000081916F018093F1002197FFEFAF1ABF0ADF
:10531000CECFFC018091EB039091EC0386179707A9
:10532000A0F06115710529F49091E8009E779093A3
:10533000E80090E06115710551F4911108C0809169
:10534000E80082FF34C080E00895BC01F2CF809174
:10535000E4038823C1F18530C1F18091E80083FD29
:1053600030C08091E80082FDEACF8091E80080FFA4
:10537000E1CF8091F3002091F200382F6115710583
:1053800019F02830310558F091E02830310509F046
:1053900090E02091E8002E772093E800CBCF819118
:1053A0008093F100615071092F5F3F4FE7CF8091EB
:1053B000E403882341F0853041F08091E80083FFC9
:1053C000BECF81E0089582E0089583E00895FC0156
:1053D0008091EB039091EC0386179707A0F061157D
:1053E000710529F48091E8008E778093E80090E0C1
:1053F0006115710551F4911108C08091E80082FF98
:1054000035C080E00895BC01F2CF8091E403882389
:10541000C9F18530C9F18091E80083FD31C08091E8
:10542000E80082FDEACF8091E80080FFE1CF809123
:10543000F3002091F200382F6115710519F0283022
:10544000310558F091E02830310509F090E0809165
:10545000E8008E778093E800CBCF84918093F100B1
:105460003196615071092F5F3F4FE6CF8091E40381
:10547000882341F0853041F08091E80083FFBDCF63
:1054800081E0089582E0089583E00895982F973091
:1054900028F08F708093E90081E008959093E900EF
:1054A000242F762F50E0981731F07091EC00209166
:1054B000ED005091F00021FD02C09F5FE8CF3091D8
:1054C000EB003E7F3093EB003091ED003D7F309359
:1054D000ED003091EB0031603093EB007093EC0005
:1054E0002093ED005093F0002091EE0027FDE5CFD2
:1054F00080E008958091E50387FF13C08091E80064
:1055000082FF06C08091E8008B778093E80004C09A
:105510008091E4038111F2CF08958091E403882300
:10552000D9F38091E80080FFF8CF8091E8008E7772
:10553000ECCF2091E4003091E50095E6A90120919F
:10554000EC00822F817020FF06C08091E80080FF70
:1055500006C080E008952091E80022FD1AC08091E5
:10556000E403882389F0853089F08091EB0085FD84
:105570000FC02091E4003091E50042175307F9F283
:105580009150E1F684E0089582E0089583E0089563
:1055900081E008950E94392B0E94412BE0EEF0E05B
:1055A000808181608083E8EDF0E080818F77808367
:1055B00019BCA7EDB0E08C918E7F8C9380818F7E9B
:1055C00080831092E30308950F931F93CF93DF938B
:1055D0000E94392B0E94412BC8EDD0E088818F7743
:1055E000888388818068888388818F7D888319BCBF
:1055F0001092E4031092E0031092E2031092E10390
:1056000000EE10E0F80180818B7F808388818160CB
:10561000888342E060E080E00E94462AE1EEF0E00C
:1056200080818E7F8083E2EEF0E0808181608083E4
:10563000808188608083F80180818E7F808388816B
:1056400080618883DF91CF911F910F910895E8EDDC
:10565000F0E080818F7E8083E7EDF0E080818160E3
:10566000808384E082BF81E08093E3030E94E42A88
:105670000895E8EDF0E080818E7F80831092E20053
:1056800008951092DA001092E10008951F920F928F
:105690000FB60F9211242F933F934F935F936F9305
:1056A0007F938F939F93AF93BF93EF93FF938091DB
:1056B000E10082FF0BC08091E20082FF07C0809171
:1056C000E1008B7F8093E1000E94FB268091DA004D
:1056D00080FF19C08091D80080FF15C08091DA004A
:1056E0008E7F8093DA008091D90080FF96C080E1A0
:1056F00089BD82E189BD09B400FEFDCF81E08093C0
:10570000E4030E94A8268091E10080FF19C08091E7
:10571000E20080FF15C08091E2008E7F8093E2005E
:105720008091E20080618093E2008091D8008062E5
:105730008093D80019BC85E08093E4030E94D726AB
:105740008091E10084FF2BC08091E20084FF27C09C
:1057500080E189BD82E189BD89B5982F917080FF74
:10576000FBCF8091D8008F7D8093D8008091E1009D
:105770008F7E8093E1008091E2008F7E8093E20033
:105780008091E20081608093E2008091E0038823B1
:1057900009F449C084E08093E4030E94E8268091E4
:1057A000E10083FF29C08091E20083FF25C0809142
:1057B000E100877F8093E10082E08093E403109210
:1057C000E0038091E1008E7F8093E1008091E20010
:1057D0008E7F8093E2008091E20080618093E200FE
:1057E00042E060E080E00E94462A8091F0008860FC
:1057F0008093F0000E94C926FF91EF91BF91AF9175
:105800009F918F917F916F915F914F913F912F91D8
:105810000F900FBE0F901F90189519BC1092E403C3
:105820000E94BE2670CF8091E30087FD93E09093A5
:10583000E403B3CF1F920F920FB60F9211242F9350
:105840003F934F935F936F937F938F939F93AF9308
:10585000BF93CF93DF93EF93FF93D091E900DF7075
:105860008091EC00C82FC17080FDC0E81092E90063
:105870008091F000877F8093F00078940E945E2CE6
:105880001092E9008091F00088608093F000CD2BA9
:10589000CF70C093E900FF91EF91DF91CF91BF915D
:1058A000AF919F918F917F916F915F914F913F91B8
:1058B0002F910F900FBE0F901F901895AAE2B0E0A5
:1058C000E4E6FCE20C94F52D85EE93E02091F100E6
:1058D000FC012193CF01F3E08D3E9F07B9F70E94B1
:1058E00056278091E80083FF1EC18091E5039091C7
:1058F000E6039A3008F017C1E92FF0E0E95EF04DB9
:105900000C94E02D803899F0823809F00CC1809118
:10591000E9038F70873008F006C18093E900809119
:10592000EB0085FB882780F91092E90006C0809182
:10593000E1039091E203911182609091E800977FDA
:105940009093E8008093F1001092F1008091E800BC
:105950008E77E5C0882309F4D3C0823009F0E3C014
:105960008091E7038111D6C08091E9038F702FEFFA
:10597000280F263008F0D7C08093E9002091EB0073
:1059800020FFC8C0933031F48091EB008062809397
:10599000EB00C0C09091EB0090619093EB0021E090
:1059A00030E001C0220F8A95EAF72093EA001092B6
:1059B000EA008091EB008860EACF8111B4C01091B9
:1059C000E7031F778091E3008078812B8093E300C9
:1059D0008091E800877F8093E8000E947A2A809176
:1059E000E80080FFFCCF8091E30080688093E300B3
:1059F00082E0111183E08093E40395C080588230E7
:105A000008F091C08091E7039091E8038C3D23E07A
:105A10009207A1F583E08A838AE289834FB7F894DD
:105A2000DE01139620E03EE051E2E32FF0E05093D8
:105A30005700E49120FF03C0E295EF703F5FEF70E5
:105A40008E2F90E0EA30C0F0C7968D939D932F5F24
:105A5000243159F74FBF8091E800877F8093E80099
:105A60006AE270E0CE0101960E9489298091E800E7
:105A70008B778093E80057C0C096E7CF6091E90329
:105A80007091EA03AE014F5F5F4F0E94C528BC01D1
:105A9000892B09F448C09091E800977F9093E80023
:105AA00089819A810E94E729E1CF8038E1F58091D0
:105AB000E800877F8093E8008091E0038093F10005
:105AC00045CF811130C09091E703923060F580910D
:105AD000E800877F8093E8009093E0030E947A2A91
:105AE0008091E003882311F084E005C08091E300F9
:105AF00087FDFACF81E08093E4030E943C2713C026
:105B00008091E703813079F481E0933009F080E0FF
:105B10008093E2031092E9008091E800877F8093F0
:105B2000E8000E947A2A8091E80083FF0AC08091F1
:105B3000E800877F8093E8008091EB00806280938B
:105B4000EB00AA96E3E00C94112ECF938091E4032E
:105B50008823A1F0C091E900CF709091EC00892FCB
:105B6000817090FD80E8C82B1092E9008091E800D8
:105B700083FD0E945E2CCF70C093E900CF91089501
:105B8000991B79E004C0991F961708F0961B881F8F
:105B90007A95C9F78095089597FB072E16F400941F
:105BA00007D077FD09D00E941D2E07FC05D03EF4DA
:105BB000909581959F4F0895709561957F4F0895B9
:105BC000EE0FFF1F0590F491E02D09942F923F9264
:105BD0004F925F926F927F928F929F92AF92BF92FD
:105BE000CF92DF92EF92FF920F931F93CF93DF93A9
:105BF000CDB7DEB7CA1BDB0B0FB6F894DEBF0FBE06
:105C0000CDBF09942A88398848885F846E847D8452
:105C10008C849B84AA84B984C884DF80EE80FD8054
:105C20000C811B81AA81B981CE0FD11D0FB6F894CA
:105C3000DEBF0FBECDBFED010895AA1BBB1B51E116
:105C400007C0AA1FBB1FA617B70710F0A61BB70BEC
:105C5000881F991F5A95A9F780959095BC01CD0191
:105C60000895FB01DC0104C08D910190801921F49D
:105C700041505040C8F7881B990B0895FB01DC0187
:105C800002C001900D9241505040D8F70895F99903
:105C9000FECF92BD81BDF89A992780B50895A8E1FD
:105CA000B0E042E050E00C948B2EDC01A40FB51F55
:105CB0004150504048F0CB01840F951F2E910E9417
:105CC000662E41505040D0F70895262FF999FECF07
:105CD00092BD81BDF89A019700B4021639F01FBA3F
:105CE00020BD0FB6F894FA9AF99A0FBE089503965C
:105CF000272F0E94662E0E94652E252F0E94662E59
:105D0000242F0C94662E0196272F0E94662E0C9449
:105D1000652EDC01CB01FC01F999FECF06C0F2BD76
:105D2000E1BDF89A319600B40D9241505040B8F759
:105D30000895F894FFCFE10AE10A310B310B960B7D
:105D4000B20B100B100BB70B280C370C370C5A1872
:105D500067186C1870187218741876187818091C5F
:105D6000EC1B121C6A1BB91CB91CE51BB91CB91C25
:105D7000421CB91C521C9F1CB91CB91CB91CB91C73
:105D8000711CB91CB91C621CB91C2B1CB91CB91C98
:105D9000B71CB71CB71CB71CB71CB71CB71CB71C6B
:105DA000B71CB11CB91C091CDA1BB91CB91CB91CE5
:105DB000B91CB91CB91CB91CB91CB91CB91CB11C43
:105DC000B91CB91CE51BB91CB51CB51CB51CB51C10
:105DD000B51CB51CB51CB51CB51CB11CAA1D1E1EDE
:105DE000B21D7C1D801DB61D841DBA1DC61D901DD3
:105DF000171E941DCA1D981DCE1DF61D9C1DD21D7B
:105E0000FD1DA21DD81DE01D881DBE1D8C1DC21DBF
:105E1000A61DDC1DEC1D061E151E761DAE1D251EC5
:105E2000802286226F227A228C2292229822822C31
:105E3000AA2C932DAA2C932DDD2CFE2C932D552DC1
:025E4000612DD2
:105E42005E037E03280850011E0A140100000100AF
:105E5200582591268A2683267C26E200E900EA005C
:105E6200B500B600B700CD008301CC008A019201D3
:105E720094012102230224022502260227022A0279
:105E8200B300B4006F0070009F01CB019F02A0021B
:105E9200818283E200E900EA00B500B600B700CDD6
:105EA200008301CC008A0192019401210223022481
:105EB200022502260227022A02B300B4006F0070F4
:105EC200009F01CB019F02A0028182839766353435
:105ED200C69436F6F79637909193923F3F3F006D06
:105EE2006B5F64656C6179006D6B5F696E7465727E
:105EF20076616C006D6B5F6D61785F737065656470
:105F0200006D6B5F74696D655F746F5F6D617800C2
:105F12006D6B5F776865656C5F6D61785F737065E7
:105F22006564006D6B5F776865656C5F74696D654C
:105F32005F746F5F6D6178000A092D205665727378
:105F4200696F6E202D0A5649443A2030783132303A
:105F5200392822546563686E6F6D616E63792229F8
:105F6200205049443A203078413145352822417445
:105F7200726575732229205645523A2030783030A6
:105F820030380A4255494C443A202028446563205F
:105F920020322032303234290A4F5054494F4E5366
:105FA2003A204C554641204D4F5553454B455920BB
:105FB20045585452414B455920434F4E534F4C453F
:105FC20020434F4D4D414E44204E4B524F203430D2
:105FD20039360A4743433A20382E332E3020415671
:105FE200522D4C4942433A20322E302E3020415617
:105FF200525F415243483A20617672350A0044B6F4
:0E600200152A0C740B5F0B0B0B240B3D0B00CF
:00000001FF
